:020000040000FA
:0400000068EF00F0B5
:08000800056ED8CF06F0E0CF31
:1000100007F00001E9CF0DF0EACF08F0E1CF09F0D9
:10002000E2CF0AF0D9CF0BF0DACF0CF0F3CF14F017
:10003000F4CF15F0FACF16F000C00FF001C010F0A9
:1000400002C011F003C012F004C013F0F2AA2CEFAA
:1000500000F0F2B44FEF00F00FC000F010C001F05C
:1000600011C002F012C003F013C004F00DC0E9FF8C
:1000700008C0EAFF088E09C0E1FF0AC0E2FF0BC01A
:10008000D9FF0CC0DAFF14C0F3FF15C0F4FF16C08F
:10009000FAFF055007C0E0FF06C0D8FF1000929499
:1000A0008994F2942CEF00F0EA6A190EE96EEF5091
:1000B0000DE0020E016E006A002EFED7012EFBD766
:1000C000970E006E002EFED7EF2EF3D7AEEF00F0A6
:1000D000F86AD09E088EEA6AE96A700ED36ED35031
:1000E000B8960C0EAF6EA20EAC6E900EAB6EC150F9
:1000F000C00B0F09C16E070EB46EC150C00B0F09C3
:10010000C16EC290B098C69A949E93809392010E4D
:10011000C66E000EC76ED190810ED56ECD6A000EF0
:10012000CA6E000ECB6EB70EB16E070EB46E925053
:10013000926E060E006E002EFED70000B450A19CF9
:10014000B56AF19EF28AC00EF212FF0E936E81CF55
:1001500018F092928972640E196EA6D7FF0E936EF4
:100160008150185C02E092948984FF0E936E81CFD7
:0601700018F0EFD70300B8
:020000040030CA
:0E0000003FC8190E008781000FC00FE00F40AF
:00000001FF
